:02000000F32FDC
:100C3A00831205118514212E222E232E242E83128F
:100C4A0005150800831205152A2E2B2E2C2E2D2E63
:100C5A0083128514302E312E322E332E83128510B4
:100C6A00362E372E382E392E080083120515851494
:100C7A003E2E3F2E402E412E83120511442E452E24
:100C8A00462E472E831285104A2E4B2E4C2E4D2E61
:100C9A00080083120511512E522E532E542E831200
:100CAA008514572E582E592E5A2E831285105D2ED2
:100CBA005E2E5F2E602E831205150800831285149E
:100CCA00831605158312051D6D2EF101F10A6E2E8C
:100CDA00F10183160511831205110630F000F00B9D
:100CEA00742E0000831285107A2E7B2E7C2E7D2E88
:100CFA0071080800F00183160515F1010310F00DC3
:100D0A0083128514882E892E8A2E8B2E831205191A
:100D1A00F00A8510902E912E922E932E0830F10A09
:100D2A007102031C842E8316051170080800F50051
:100D3A00F601740876020318B82E1D263A2675089D
:100D4A00B9266326003A031DB82E7208B92663260F
:100D5A00003A031DB82E7308B9266326003A031D0C
:100D6A00B82EF60A9E2E1D2EF000F101F01FC02E9D
:100D7A0083120515C22E83120511C32EC42EC52E49
:100D8A00C62E83128514C92ECA2ECB2ECC2E8312C0
:100D9A00851007307106031905110310F00DD52EC1
:100DAA00D62ED72ED82E0830F10A71020318080061
:100DBA00BB2EF6003A267608B9266326003A031DAA
:100DCA00212F7208B9266326003A031D212F3A26DD
:100DDA0076080138B9266326003A031D212F8316A7
:100DEA000515F701F8017808803AF400803074029A
:100DFA00031D012F730877020318212F7F26831200
:100E0A00A40083160511092F0A2F0B2F0C2F730824
:100E1A00FF3EF400FF3003180030F5007806031D8A
:100E2A00182F7708740603191C2F4E261D2F272604
:100E3A00F70A0319F80AF82E1D2E831605118510D4
:100E4A000510FF309C009B0086019E009D008312C6
:100E5A00860083160614831205141530FB004B30E6
:100E6A00FA00BE30F900F90B382FFA0B382FFB0BBA
:100E7A00382F00001530FB004B30FA00BE30F90065
:100E8A00F90B452FFA0B452FFB0B452F0000FC01F0
:100E9A001330F2009B30E8279C260D30F900F90B3D
:100EAA00542F1330F200E230F301F30ADE260D303C
:100EBA00F900F90B5E2F0530FC0A7C02031C4D2F4A
:100ECA002430F2000330E8279C260430F200203058
:100EDA00E8279C261030F2002030E8279C260330B1
:100EEA00F2004530E8279C261C30F2002130E82722
:100EFA009C261130F2001030E8279C261830F200A8
:100F0A008030E8279C261930ED279C261A30F200FB
:100F1A005530E8279C261B30F200E230F301F30A31
:100F2A00F401F40A9C261D30ED279C261E30F2009F
:100F3A007130E8279C261F30F2000230E8279C26F1
:100F4A002030F2008030E8279C262130F2003E3023
:100F5A00E8279C262230ED279C262330F2000C300D
:100F6A00E8279C261530FB004B30FA00BE30F9000A
:100F7A00F90BBD2FFA0BBD2FFB0BBD2F000015304F
:100F8A00FB004B30FA00BE30F900F90BCA2FFA0BFE
:100F9A00CA2FFB0BCA2F00001530FB004B30FA009A
:100FAA00BE30F900F90BD72FFA0BD72FFB0BD72F2F
:100FBA00000083120510073083169F0063000000AB
:100FCA0000000000E02FF300E230F401F40A080008
:100FDA00F200E230F301F401F40A0800A130A000A3
:100FEA00A030A1000130A2000430A300E230FD00CD
:060FFA00A4018301222F77
:06400000E33F5D3FF03FCD
:00000001FF
